:100000000C9466010C948E010C948E010C948E015C
:100010000C948E010C948E010C948E010C948E0124
:100020000C948E010C948E010C948E010C948E0114
:100030000C948E010C948E010C948E010C948E0104
:100040000C94BC220C948E010C94CE240C941C2590
:100050000C948E010C948E010C948E010C948E01E4
:100060000C948E010C948E013C76657273696F6EF0
:1000700020302E393430393E0046726565205241B9
:100080004D3A20004552524F523A20005379732086
:10009000766F6C74733A200053797320766F6C74AA
:1000A00073206368617267696E673A2000537973E1
:1000B00020766F6C74732069646C653A200062610D
:1000C0007474506C757350696E204F4E0062617489
:1000D00074506C757350696E204F4646006375729C
:1000E00072656E745A65726F4F66667365743A0016
:1000F00053616D706C652073697A653A20003E002B
:1001000020002000200020002000200020002000EF
:1001100020003C0041444A555354494E4720006159
:10012000646A416D70735F4F4E200061646A566F60
:100130006C74735F4F4E200063656C6C5368756E12
:1001400074335F4F4E200063656C6C5368756E743A
:10015000325F4F4E200063656C6C5368756E74316E
:100160005F4F4E200074617267657420416D70733B
:100170003A200074617267657420566F6C74733A2C
:10018000200070777250574D3A200049444C45206A
:10019000544F54414C20566F6C74733A20004944BC
:1001A0004C4520566F6C747320333A200049444C00
:1001B0004520566F6C747320323A200049444C45F8
:1001C00020566F6C747320313A20004348415247E7
:1001D000494E4720544F54414C20566F6C74733A2B
:1001E00020004348415247494E4720566F6C747374
:1001F00020333A20004348415247494E4720566F2A
:100200006C747320323A20004348415247494E47AC
:1002100020566F6C747320313A2000434841524796
:10022000494E472063757272656E7420414D50537C
:100230003A2000544F54414C20766F6C74733A202E
:1002400000766F6C747320333A2000766F6C747391
:1002500020323A2000766F6C747320313A200043CC
:10026000757272656E7420416D70733A20000000E3
:100270000000240027002A000000000025002800BC
:100280002B000000000023002600290004040404C1
:100290000404040402020202020203030303030330
:1002A000010204081020408001020408102001020D
:1002B00004081020000000070002010000030406EB
:1002C00000000000000000009F02882611241FBECD
:1002D000CFEFD8E0DEBFCDBF15E0A0E0B1E0ECE0AD
:1002E000F8E502C005900D92A030B107D9F716E0ED
:1002F000A0E0B5E001C01D92AB38B107E1F712E014
:10030000CCECD2E004C02297FE010E94002CC83C35
:10031000D107C9F70E94BE240C94042C0C94000051
:10032000EF92FF920F931F937A018B01AA2797FDFB
:10033000A095BA2FBC01CD010E947B2AA80197018C
:100340000E942F2B20E030EC4FE754E40E94E0297C
:1003500020E030E040E250E40E94772924EA30E7D0
:100360004DE35EE30E94E0291F910F91FF90EF9013
:1003700008956F927F928F929F92AF92BF92CF9289
:10038000DF92EF92FF920F931F933A014B0181305E
:10039000910599F4222389F0A0906705B090680533
:1003A000C0906905D0906A0520916B0530916C056D
:1003B00040916D0550916E0515C082309105D9F4BC
:1003C0002223C9F0A0906B05B0906C05C0906D051C
:1003D000D0906E05209167053091680540916905C0
:1003E00050916A05E0906F05F090700500917105DD
:1003F000109172056EC083309105D9F42223C9F0A3
:10040000A0906F05B0907005C0907105D0907205F6
:1004100020916705309168054091690550916A0502
:10042000E0906B05F0906C0500916D0510916E05E4
:1004300050C08130910599F4222389F4A09077056A
:10044000B0907805C0907905D0907A0520917B0511
:1004500030917C0540917D0550917E0515C082301C
:100460009105D9F42223C9F4A0907B05B0907C05B6
:10047000C0907D05D0907E0520917705309178055C
:100480004091790550917A05E0907F05F0908005C4
:1004900000918105109182051CC00397D1F422239D
:1004A000C1F4A0907F05B0908005C0908105D090E8
:1004B000820520917705309178054091790550911A
:1004C0007A05E0907B05F0907C0500917D05109108
:1004D0007E05C601B5010E947729A40193010E94FF
:1004E0002B2B1816ECF0C601B501A80197010E944C
:1004F0007729A40193010E942B2B181614F010E009
:1005000010C010E0C601B5012091E9043091EA0461
:100510004091EB045091EC040E942B2B18160CF424
:1005200011E0812F1F910F91FF90EF90DF90CF90FE
:10053000BF90AF909F908F907F906F900895609143
:10054000C6047091C7048091C8049091C9042DEC31
:100550003CEC4CE45DE30E94772960933205709394
:1005600033058093340590933505089585E696E02C
:1005700068E670E00E9452270895DF92EF92FF92A2
:100580000F931F93482FD92E8B0183EDE82E85E022
:10059000F82EC7010E94B0220F5F1F4FC701B8019C
:1005A0004D2D0E94B0221F910F91FF90EF90DF9090
:1005B0000895609157057091580580915905909163
:1005C0005A0520915B0530915C0540915D05509185
:1005D0005E050E94782920915F0530916005409169
:1005E0006105509162050E9478299B01AC016091E0
:1005F00063057091640580916505909166050E9480
:100600002B2B181624F58091E7049091E8040197AC
:1006100031F180919A0590919B05823091058CF083
:1006200010929B0510929A0581E090E09093E80467
:100630008093E70485E696E060E071E00E9464291B
:100640000895019690939B0580939A0508951092C2
:100650009B0510929A051092E8041092E704089501
:10066000EF92FF920F931F939C018130910539F116
:10067000823091051CF4009749F0FFC0823091054B
:10068000B9F18330910509F0F8C085C08091BF05AC
:100690009091C005892B09F4F0C080918C05909150
:1006A0008D05892B09F0E9C01092C0051092BF0595
:1006B0001092BE051092BD058DE060E0DCC0809117
:1006C000BF059091C005019709F4D7C080918C05B2
:1006D00090918D05892B09F0D0C03093C0052093EF
:1006E000BF053093BE052093BD058DE061E0C3C01A
:1006F0002091B9053091BA054091BB055091BC05D8
:10070000211531054105510531F08091BF059091CA
:10071000C005029779F082E090E09093C005809345
:10072000BF0581E090E09093BE058093BD058DE00C
:1007300061E022C08091000590910105A091020521
:10074000B091030582179307A407B50708F495C075
:100750008091BD059091BE05019729F41092BE05C8
:100760001092BD0506C081E090E09093BE05809395
:10077000BD058DE06091BD050E946A248091000551
:1007800090910105A0910205B0910305845D9E4FF3
:10079000AF4FBF4F36C080918C0590918D05892B4E
:1007A00009F06BC0E090B905F090BA050091BB0567
:1007B0001091BC05E114F1040105110531F080919F
:1007C000BF059091C005039729F183E090E09093D5
:1007D000C0058093BF0581E090E09093BE058093B3
:1007E000BD058DE061E00E946A2480910005909132
:1007F0000105A0910205B09103058A5B9F4FAF4FA1
:10080000BF4F8093B9059093BA05A093BB05B093F1
:10081000BC0533C0209100053091010540910205CF
:10082000509103052E153F054007510730F1809187
:10083000BD059091BE05019749F41092BE05109236
:10084000BD0524523A4F4F4F5F4F0AC081E090E000
:100850009093BE058093BD052A5B3F4F4F4F5F4F7E
:100860002093B9053093BA054093BB055093BC055E
:100870008DE06091BD050E946A241F910F91FF9049
:10088000EF90089582E061E00E946A241092ED04E6
:1008900080918B05882331F085E696E06CE071E06D
:1008A0000E946429089582E060E00E946A24809199
:1008B000ED04882351F480918B05882331F085E67F
:1008C00096E064E271E00E94642981E08093ED0487
:1008D000089583E061E00E946A2480918B0588235B
:1008E00031F085E696E06EE371E00E946429089598
:1008F0008130910589F4662341F088E061E00E942F
:100900006A2481E080934205089588E060E00E94B7
:100910006A241092420508958230910589F4662375
:1009200041F087E060E00E946A2481E08093430503
:10093000089587E061E00E946A24109243050895BB
:10094000039781F4662341F084E060E00E946A240A
:1009500081E080934405089584E061E00E946A2468
:100960001092440508958DE061E00E946A2460E0E1
:100970007DE780E090E00E9412238DE060E00E941D
:100980006A2460E07DE780E090E00E9412238DE021
:1009900061E00E946A2460E07DE780E090E00E94D0
:1009A00012238DE060E00E946A2460E07DE780E031
:1009B00090E00E9412238DE061E00E946A2460E0D2
:1009C0007DE780E090E00E9412238DE060E00E94CD
:1009D0006A2460E07DE780E090E00E9412230895A1
:1009E000DF92EF92FF920F931F938C0193EDE92E0C
:1009F00095E0F92EC701B8010E94A922D82E0F5FF9
:100A00001F4FC701B8010E94A9226D2D0E94DE264A
:100A10001F910F91FF90EF90DF900895FF920F9339
:100A20001F93CF93DF9385E696E064E571E00E9423
:100A300067288091DB049091DC04069721F0FF2465
:100A4000C6E0D0E01BC085E696E062E671E039C002
:100A5000CE010E94F0048C01FF2031F085E696E083
:100A600065E671E00E94672885E696E0B8014AE0F5
:100A700050E00E9435282296FF24F3948091DB04F5
:100A80009091DC040197C817D90714F380918C0565
:100A900090918D050817190781F085E696E065E6C7
:100AA00071E00E94672860918C0570918D0585E644
:100AB00096E04AE050E00E94352885E696E067E639
:100AC00071E00E946429DF91CF911F910F91FF90F7
:100AD000089510921C0510921B0585E060E070E0FF
:100AE0000E94CB23109219051092180510921A0536
:100AF00085E090E09093B9048093B80408950E9433
:100B0000690581E090E060E00E94780482E090E076
:100B100060E00E94780483E090E060E00E94780446
:100B200008950E947F051092290580E090E00E94C0
:100B3000300308952F923F924F925F926F927F926F
:100B40008F929F92AF92BF92CF92DF92EF92FF92DD
:100B50000F931F93CF93DF93EC010F2EF3E32F2E10
:100B6000F3E33F2EF3E74F2EF0E45F2EF02D0F2E30
:100B7000F0E06F2EF0E07F2EF0E68F2EF0E49F2E57
:100B8000F02D0F2EFDECAF2EFCECBF2EFCE5CF2E92
:100B9000F0E4DF2EF02D0F2EF0E0EF2EF0E0FF2E30
:100BA000F0E00F2FFFE31F2FF02D80918C05909127
:100BB0008D05C817D90761F1209751F16091DB04C9
:100BC0007091DC04CE010E94BD026091DB04709143
:100BD000DC046E5F7F4F80E090E00E94BD02809158
:100BE000DB049091DC0402969093DC048093DB0498
:100BF00080918B05882331F085E696E069E671E007
:100C00000E946429D0938D05C0938C050E940E0527
:100C1000D0938D05C0938C0582E090E00E94300354
:100C200020918C0530918D052115310529F480E046
:100C300090E00E94300353C0243131050CF44FC0C2
:100C4000C9014497449768F0C9018897449728F4EC
:100C50001092DA040E94910542C0C901CC974497D2
:100C600078F50E94910586E696E6A6E7B0E48093C3
:100C7000C6049093C704A093C804B093C9042092FB
:100C8000320530923305409234055092350560921A
:100C9000D6047092D7048092D8049092D904A0927E
:100CA000E904B092EA04C092EB04D092EC04E09222
:100CB000CA04F092CB040093CC041093CD040FC06F
:100CC000205530402431310550F41092DA040E944E
:100CD000910585E696E061E871E00E9464298091C3
:100CE000DB049091DC044697F4F00E94A60688236A
:100CF000D1F4A6E0B0E0B093DC04A093DB048091D3
:100D00008C0590918D0566E070E00E94BD02809197
:100D1000DB049091DC0402969093DC048093DB0466
:100D2000CEE3D0E042CFDF91CF911F910F91FF90A2
:100D3000EF90DF90CF90BF90AF909F908F907F907B
:100D40006F905F904F903F902F900895CF93DF93D7
:100D5000C6E0D0E008C0CE010E94F004889714F0ED
:100D600080E025C022968091DB049091DC048C17F2
:100D70009D078CF7C6E0D0E007C083ED95E0BE018B
:100D800040E00E94B02221968091DB049091DC0427
:100D900001968C179D078CF786E090E09093DC0419
:100DA0008093DB0480E090E00E949A0581E0DF916F
:100DB000CF91089560915305709154058091550528
:100DC000909156052091CA043091CB044091CC04F7
:100DD0005091CD040E94772929E23CE54FE05EE383
:100DE0000E942B2B181694F48091AF059091B005BA
:100DF000853191052CF083E590E00E949A0506C0AC
:100E000001969093B0058093AF0508951092B005B8
:100E10001092AF050895609153057091540580912B
:100E200055059091560520E030E040E05FE30E94D8
:100E3000DC298823CCF480911B0590911C05843B10
:100E4000910591F48091AD059091AE0585319105A4
:100E50002CF08AE290E00E949A0506C001969093D9
:100E6000AE058093AD0508951092AE051092AD05C4
:100E700008956091530570915405809155059091A6
:100E800056052DEC3CEC4CE45EE30E942B2B18162F
:100E9000D4F480911B0590911C05892BA1F48091BD
:100EA000A7059091A805853091053CF082E590E07A
:100EB0000E949A050E94530406C001969093A805CB
:100EC0008093A70508951092A8051092A70508958C
:100ED00083E060E00E946A2480918B05882331F0D2
:100EE00085E696E060E971E00E9464298091E5045E
:100EF0009091E604019751F060E072EE84E090E09A
:100F00000E9412238DE390E00E949A050895AF920B
:100F1000BF92CF92DF92EF92FF920F931F931092A6
:100F2000B5051092B6051092B7051092B8058091DC
:100F3000ED048823B9F080911B0590911C051816CB
:100F4000190684F0609163057091640580916505D0
:100F50009091660520E030E040E651E40E94DC29F3
:100F600088231CF481E090E04DC0A090B105B090C2
:100F7000B205C090B305D090B4056091530570914F
:100F800054058091550590915605A60195010E9442
:100F900077299B01AC0168E17AEF88E29BEB0E9424
:100FA00077297B018C016093B1057093B205809322
:100FB000B3059093B40520E030E040E050E00E949B
:100FC0002B2B18165CF4C801B70120E030E040E894
:100FD0005EE30E942B2B18165CF017C0C801B70106
:100FE00020E030E040E85EEB0E94DC2988236CF4CE
:100FF000A092B105B092B205C092B305D092B405EB
:1010000081E590E00E949A0548C080918B05882375
:1010100041F185E696E067EA71E00E946429C60125
:10102000B5012091B1053091B2054091B3055091C1
:10103000B4050E94DC298823A1F085E696E066EBE2
:1010400071E00E9467284091B1055091B20560910E
:10105000B3057091B40585E696E022E030E00E9489
:1010600051296091B1057091B2058091B3059091BD
:10107000B40520E030E04AE754E40E942F2B20E042
:1010800030E04AE754E40E9478290E94482ADC01B3
:10109000CB0164E070E00E94BD021F910F91FF90B0
:1010A000EF90DF90CF90BF90AF9008958091E504CE
:1010B0009091E604019771F5609163057091640564
:1010C000809165059091660526E636E646E551E491
:1010D0000E94DC298823F4F48091A5059091A6054F
:1010E0008A3091058CF01092A6051092A50585E630
:1010F00096E068EC71E00E9464290E94910584E00A
:1011000090E00E949A05089501969093A605809319
:10111000A50508951092A6051092A5050895609161
:101120005705709158058091590590915A05209165
:101130005B0530915C0540915D0550915E050E9414
:1011400078292DEC3CEC4CE45EE30E94DC298823FA
:101150003CF483E090E00E949A050E949105089576
:1011600080918C0590918D05039721F480E090E0AB
:101170000E949A0508958091A2058823F9F40E949F
:10118000910585E696E061ED71E00E946429809109
:10119000000590910105A0910205B09103058053CF
:1011A000984FAF4FBF4F80939C0590939D05A093A0
:1011B0009E05B0939F0581E08093A2050895EF926C
:1011C000FF920F931F938091E5049091E604892B81
:1011D00009F0F9C0E090E904F090EA040091EB0412
:1011E0001091EC0460915705709158058091590554
:1011F00090915A05A80197010E94DC2987FD1CC027
:1012000060915B0570915C0580915D0590915E0534
:10121000A80197010E94DC2987FD0EC060915F053F
:10122000709160058091610590916205A801970118
:101230000E94DC2988239CF58091A0059091A1054E
:101240008035910534F11092A1051092A0050E94FD
:10125000BB086091E9047091EA048091EB049091DD
:10126000EC042DEC3CEC4CE450E40E94DC29882397
:10127000D1F486E190E00E949A0580918B05882345
:1012800009F4A1C085E696E06CED71E00E94642946
:101290009AC001969093A1058093A00504C0109276
:1012A000A1051092A0056091570570915805809195
:1012B000590590915A0520E030E040E650E40E9444
:1012C000DC2987FD21C060915B0570915C058091F0
:1012D0005D0590915E0520E030E040E650E40E941C
:1012E000DC2987FD11C060915F05709160058091D8
:1012F00061059091620520E030E040E650E40E94F4
:10130000DC2988230CF05BC08091A3059091A40593
:10131000803591050CF44DC01092A4051092A305E0
:101320008091BF059091C0050397F1F16091DD04B4
:101330007091DE048091DF049091E00420918E058D
:1013400030918F0540919005509191050E94772929
:1013500023E333E343E75FE30E94E0296093DD0486
:101360007093DE048093DF049093E0040E94482A87
:10137000DC01CB0162E070E00E94BD026091DD04FF
:101380007091DE048091DF049091E0042DEC3CEC40
:101390004CE45DE30E942F2B60938E0570938F05C4
:1013A000809390059093910583E090E00E94300334
:1013B0000AC001969093A4058093A30504C01092DF
:1013C000A4051092A3051F910F91FF90EF9008952F
:1013D000EF92FF920F931F936091570570915805FC
:1013E0008091590590915A0520915B0530915C05DB
:1013F00040915D0550915E050E94782920915F051E
:101400003091600540916105509162050E947829F4
:101410007B018C016091D6047091D7048091D8042F
:101420009091D90420E030E040E450E40E942F2B5A
:101430009B01AC01C801B7010E94DC298823ACF4F0
:101440006091C6047091C7048091C8049091C9044A
:101450002DEC3CEC44E850E40E94DC29882329F47C
:101460008DE290E00E949A0528C00E94910560914B
:10147000C6047091C7048091C8049091C9042DECF2
:101480003CEC44E850E40E94DC298823B1F48091CC
:10149000DD049091DE04A091DF04B091E00480931C
:1014A0008E0590938F05A0939005B093910585E6E6
:1014B00096E061EF71E00E9464291F910F91FF9007
:1014C000EF900895EF92FF920F931F937B018C0191
:1014D00080918C0590918D05039749F181E080936F
:1014E00029050E947F058091000590910105A0913A
:1014F0000205B09103058E0D9F1DA01FB11F8C53D7
:10150000964FAF4FBF4F80932A0590932B05A09322
:101510002C05B0932D05845C9940A040B040809389
:10152000360590933705A0933805B09339051F9180
:101530000F91FF90EF900895EF92FF920F931F93FA
:10154000E0906305F09064050091650510916605D3
:10155000C801B70120E030E040E651E40E942B2BA7
:1015600088230CF488C010929705109296058091FC
:10157000E5049091E604019709F4EAC0809198058A
:1015800090919905823091050CF46FC010929905E5
:101590001092980581E090E09093E6048093E50432
:1015A00085E696E06BEF71E00E9464298091DA0491
:1015B000882309F4CDC0E0903205F0903305009106
:1015C000340510913505609157057091580580914B
:1015D000590590915A05A80197010E942B2B882349
:1015E000FCF060915B0570915C0580915D059091C8
:1015F0005E05A80197010E942B2B88238CF0609137
:101600005F05709160058091610590916205A80168
:1016100097010E942B2B88231CF00E94E80998C098
:1016200080918B05882331F085E696E064E072E0D6
:101630000E94642960E177E280E090E00E94620A03
:101640008091000590910105A0910205B0910305DC
:1016500088579C4EAF4FBF4F8093B5059093B6050A
:10166000A093B705B093B80573C001969093990500
:10167000809398056DC0109299051092980560911D
:101680005705709158058091590590915A05209100
:101690005B0530915C0540915D0550915E050E94AF
:1016A000782920915F053091600540916105509146
:1016B00062050E9478299B01AC01C801B7010E9414
:1016C000DC2918160CF440C0109299051092980568
:1016D0008091E5049091E604892BD1F180919605E3
:1016E00090919705823091054CF1109297051092D8
:1016F00096051092E6041092E50485E696E063E113
:1017000072E00E9464290E9442041092B505109272
:10171000B6051092B7051092B8058091DA048823B7
:10172000B9F080918B05882331F085E696E06EE173
:1017300072E00E9464290E9491050AC0019690936C
:1017400097058093960504C0109297051092960510
:101750001F910F91FF90EF9008952F923F924F921B
:101760005F926F927F928F929F92AF92BF92CF9231
:10177000DF92EF92FF920F931F93DF93CF9300D0EE
:1017800000D0CDB7DEB78091000590910105A09102
:101790000205B091030589839A83AB83BC83809350
:1017A000140590931505A0931605B0931705809125
:1017B00018058823D9F06090B0047090B10480902F
:1017C000B2049090B304A0903E05B0903F05C09045
:1017D0004005D09041050F2EFAE02F2EF7ED3F2E59
:1017E000F3EA4F2EFCE35F2EF02D1AC06090B40494
:1017F0007090B5048090B6049090B704A0908705CF
:10180000B0908805C0908905D0908A050F2EF9E226
:101810002F2EFCE53F2EFFE84F2EFDE35F2EF02D2F
:10182000C601B501A40193010E9477297B018C01B7
:1018300020E030E040E050E00E942B2B181624F00E
:1018400017FB109517F91095C801B701A201910176
:101850000E942B2B88230CF4F7C080911A05882353
:1018600009F04AC081E080931A0589819A81AB8191
:10187000BC8180931F0590932005A0932105B09310
:101880002205C601B501A40193010E94DC29882329
:101890001CF481E090E002C08FEF9FEF90931E0553
:1018A00080931D05C201B10120E030E040E850E422
:1018B0000E942F2B9B01AC01C801B7010E942B2B6A
:1018C00018161CF485E090E002C081E090E090934F
:1018D000B9048093B80420911D0530911E058091B4
:1018E000B8049091B904D901A89F9001A99F300D27
:1018F000B89F300D11244EC0C601B501A40193015B
:101900000E94DC298823BCF480911D0590911E055E
:101910008F5F9F4F81F481E090E09093B9048093B2
:10192000B80490931E0580931D0580911B0590912E
:101930001C05019635C0C601B501A40193010E94A2
:101940002B2B1816BCF480911D0590911E0581303B
:10195000910581F49093B9048093B8048FEF9FEFC1
:1019600090931E0580931D0580911B0590911C0589
:10197000019716C020911D0530911E058091B80475
:101980009091B904F901E89F9001E99F300DF89F0B
:10199000300D112480911B0590911C05820F931F1F
:1019A00090931C0580931B0580911B0590911C054D
:1019B000853B91053CF084EB90E090931C0580936F
:1019C0001B0506C097FF04C010921C0510921B0552
:1019D00060911B0570911C0585E00E94CB2320912E
:1019E0000005309101054091020550910305809159
:1019F000BE049091BF04A091C004B091C104820FB5
:101A0000931FA41FB51F8093080590930905A09309
:101A10000A05B0930B0580ED97E0A0E0B0E080935D
:101A2000BA049093BB04A093BC04B093BD042853A4
:101A30003F4F4F4F5F4F2093230530932405409332
:101A400025055093260502C010921A050F900F909D
:101A50000F900F90CF91DF911F910F91FF90EF901A
:101A6000DF90CF90BF90AF909F908F907F906F90BE
:101A70005F904F903F902F90089560911B0570915B
:101A80001C0585E00E94CB232091000530910105C3
:101A900040910205509103058091BE049091BF04CE
:101AA000A091C004B091C104820F931FA41FB51F61
:101AB0008093080590930905A0930A05B0930B0540
:101AC00080ED97E0A0E0B0E08093BA049093BB046F
:101AD000A093BC04B093BD0428533F4F4F4F5F4FBA
:101AE0002093230530932405409325055093260524
:101AF00010921A0508958F929F92AF92BF92CF9243
:101B0000DF92EF92FF920F931F93E0900005F09009
:101B1000010500910205109103058091C204909186
:101B2000C304A091C404B091C504A8019701281B67
:101B3000390B4A0B5B0B80912E0590912F05A091DC
:101B40003005B091310582179307A407B50708F057
:101B5000F1C0E0922E05F0922F050093300510930E
:101B6000310584EC99E0A0E0B0E08093C20490934A
:101B7000C304A093C404B093C504A0904205909000
:101B800043058090440581E090E04DEC5CEC6CE412
:101B90007DE321E00E94B901B82E882311F0BB2417
:101BA000B39482E090E04DEC5CEC6CE47DE321E0EA
:101BB0000E94B901C82E882311F0CC24C39483E07D
:101BC00090E04DEC5CEC6CE47DE321E00E94B90117
:101BD000D82E882311F0DD24D394BB2041F1E0906E
:101BE0006705F09068050091690510916A05C801C4
:101BF000B70120916B0530916C0540916D055091B6
:101C00006E050E94DC29882374F4C801B701209175
:101C10006F053091700540917105509172050E94D9
:101C2000DC2987FD04C081E090E061E003C081E031
:101C300090E060E00E947804CC2041F1E0906B05D8
:101C4000F0906C0500916D0510916E05C801B7010B
:101C500020916705309168054091690550916A05AA
:101C60000E94DC29882374F4C801B70120916F0514
:101C70003091700540917105509172050E94DC29E8
:101C800087FD04C082E090E061E003C082E090E064
:101C900060E00E947804DD2041F1E0906F05F09053
:101CA00070050091710510917205C801B70120916E
:101CB0006705309168054091690550916A050E9459
:101CC000DC29882374F4C801B70120916B05309199
:101CD0006C0540916D0550916E050E94DC2987FDD1
:101CE00004C083E090E061E003C083E090E060E046
:101CF0000E947804BB2021F4CC2011F4DD2061F097
:101D000080E29EE4A0E0B0E08093C2049093C3041C
:101D1000A093C404B093C504809142058A1541F490
:101D200080914305891521F480914405881511F0AF
:101D30000E943D0D1F910F91FF90EF90DF90CF908B
:101D4000BF90AF909F908F900895EF92FF920F9366
:101D50001F93E0900005F09001050091020510919D
:101D60000305E0922A05F0922B0500932C051093B1
:101D70002D058091360590913705A0913805B091D9
:101D80003905A8019701281B390B4A0B5B0B809181
:101D9000CE049091CF04A091D004B091D1048217C9
:101DA0009307A407B50778F480918B05882331F059
:101DB00085E696E06EE272E00E9464290E94910539
:101DC0008EE290E03BC080918C0590918D05039749
:101DD00019F40E94910566C16091670570916805CC
:101DE0008091690590916A0524EA30E745E850E45E
:101DF0000E942B2B181604F160916B0570916C05F5
:101E000080916D0590916E0524EA30E745E850E435
:101E10000E942B2B181684F060916F05709170054D
:101E2000809171059091720524EA30E745E850E40D
:101E30000E942B2B18162CF48BE290E00E949A053E
:101E400031C16091870570918805809189059091D5
:101E50008A052DEC3CEC4CE45EE30E94DC298823EF
:101E600004F5809118058823E1F080913A0590915E
:101E70003B05A0913C05B0913D05E81AF90A0A0B13
:101E80001B0B8091D2049091D304A091D404B09103
:101E9000D5048E159F05A007B10758F40E94E809E4
:101EA00001C1E0923A05F0923B0500933C05109386
:101EB0003D0581E090E00E943003E090CA04F0907C
:101EC000CB040091CC041091CD0460916705709112
:101ED00068058091690590916A052DEC3CEC4CE415
:101EE00050E40E94DC2987FD20C060916B05709151
:101EF0006C0580916D0590916E052DEC3CEC4CE4E9
:101F000050E40E94DC2987FD10C060916F0570913C
:101F1000700580917105909172052DEC3CEC4CE4BC
:101F200050E40E94DC298823A4F580918B05882346
:101F300031F085E696E060E472E00E9464298091C9
:101F4000000590910105A0910205B0910305209133
:101F50003605309137054091380550913905821B7F
:101F6000930BA40BB50B815A9B4BAD40B04018F0BE
:101F70008DE290E063CF85E090E00E949A050F2EFD
:101F8000FAE9EF2EF9E9FF2EF9E90F2FFEE31F2FF3
:101F9000F02DC801B70129E23CE54FE05EE30E9465
:101FA00077299B01AC01609187057091880580912C
:101FB000890590918A050E942B2B8823E4F160917A
:101FC0003E0570913F0580914005909141052AE0C2
:101FD00037ED43EA5CE30E9478292091C6043091F2
:101FE000C7044091C8045091C9040E94DC29181606
:101FF00014F16091B4047091B5048091B60490918D
:10200000B704A80197010E94DC29882321F480915C
:102010001905882311F40E943D0DE092B404F0925A
:10202000B5040093B6041093B70481E080931905BA
:102030001092180531C06091C6047091C704809158
:10204000C8049091C9042AE037ED43E25CE30E94A2
:1020500077297B018C016091B0047091B10480916B
:10206000B2049091B304A80197010E94DC2988234F
:1020700021F480911805882311F40E943D0DE0920F
:10208000B004F092B1040093B2041093B30481E061
:10209000809318051092190580911A05882311F470
:1020A0000E947B0D1F910F91FF90EF9008952F924A
:1020B0003F924F925F926F927F928F929F92AF92D8
:1020C000BF92CF92DF92EF92FF920F931F93CF9325
:1020D000DF93609145057091460580914905909187
:1020E0004A050E94B52BCB016093490590934A05A0
:1020F0004FE652E163E870E40E9490012091B1053F
:102100003091B2054091B3055091B4050E947829F1
:10211000609353057093540580935505909356052D
:1021200020E030E040E650EC0E94DC29882334F4C3
:1021300085E696E062E572E00E94642960915305AD
:1021400070915405809155059091560520E030E03E
:1021500040E850EC0E94DC29882334F482E090E0CF
:102160000E949A050E94680720910C0530910D0588
:1021700040910E0550910F0521153105410551057E
:1021800009F44CC060910005709101058091020531
:1021900090910305621B730B840B950B0E94792AA7
:1021A00020E03AEB4BE55AE40E94E02920915305E8
:1021B0003091540540915505509156050E942F2BA2
:1021C00020E030E04AE754E40E942F2B20918E0556
:1021D00030918F0540919005509191050E9478298A
:1021E00060938E0570938F05809390059093910571
:1021F000E090DD04F090DE040091DF041091E00433
:10220000A80197010E942B2B181644F4E0928E052A
:10221000F0928F050093900510939105C0914505AC
:10222000D091460580914B0590914C05BE010E94CE
:10223000B52B882777FD8095982F0E947B2A20E078
:1022400030EC4FE754E40E94E0292FE632E143E806
:1022500050E40E942F2B2AEF39E146E55FE30E940C
:10226000E02920E030E040E050E00E9478291B01A6
:102270002C016093570570935805809359059093EE
:102280005A0580914D0590914E05BE010E94B52BD7
:10229000882777FD8095982F0E947B2A20E030ECDC
:1022A0004FE754E40E94E0292FE632E143E850E48E
:1022B0000E942F2B21EE3FE641EE5EE30E94E029D3
:1022C000A20191010E94772920E030E040E050E037
:1022D0000E9478293B014C0160935B0570935C057B
:1022E00080935D0590935E05C201B101A401930145
:1022F0000E9478297B018C0180914F0590915005B7
:10230000BE010E94B52B882777FD8095982F0E94EB
:102310007B2A20E030EC4FE754E40E94E0292FE6CE
:1023200032E143E850E40E942F2B2FEF35EE42E9D3
:102330005EE30E94E029A80197010E94772920E02E
:1023400030E040E050E00E9478295B016C0160932E
:102350005F05709360058093610590936205C801E5
:10236000B701A60195010E9478297B018C0120917B
:10237000E1043091E2044091E3045091E4040E94AE
:10238000DC29882344F4E092E104F092E204009313
:10239000E3041093E4048091510590915205BE012D
:1023A0000E94B52B882777FD8095982F0E947B2A65
:1023B00020E030EC4FE754E40E94E0292FE632E1C0
:1023C00043E850E40E942F2B27E53FE348E65EE315
:1023D0000E94E0297B018C01CB01D8018093630529
:1023E00090936405A0936505B093660510924A0525
:1023F0001092490510924C0510924B0510924E0513
:1024000010924D051092500510924F0510925205F2
:1024100010925105D0934805C09347051092460588
:102420001092450580912805882309F408C1809100
:102430002705882321F12092670530926805409294
:10244000690550926A0560926B0570926C058092E6
:102450006D0590926E05A0926F05B0927005C092C6
:102460007105D09272058E2D80937305909374053B
:10247000A0937505B093760510922705E0C02092D1
:102480007705309278054092790550927A056092EE
:102490007B0570927C0580927D0590927E05A092CE
:1024A0007F05B0928005C0928105D0928205C70158
:1024B000D8018093830590938405A0938505B093FC
:1024C00086058091530590915405A0915505B091D2
:1024D00056058093870590938805A0938905B0934E
:1024E0008A05C201B101A40193010E942B2B88230C
:1024F0008CF0C201B101A60195010E942B2B88230B
:102500004CF020923E0530923F054092400550929B
:10251000410521C0C401B301A20191010E942B2BEE
:1025200088238CF0C401B301A60195010E942B2BD6
:1025300088234CF060923E0570923F0580924005E2
:102540009092410508C0A0923E05B0923F05C0920E
:102550004005D09241056091C6047091C7048091F6
:10256000C8049091C9042AE037ED43E25DE30E947C
:1025700078299B01AC0160913E0570913F058091E7
:102580004005909141050E942B2B1816FCF4809178
:1025900029058823D9F080911B0590911C0505978A
:1025A00090931C0580931B0597FF04C010921C0597
:1025B00010921B050E943D0D80918B05882331F000
:1025C00085E696E061E672E00E94642960918705E5
:1025D000709188058091890590918A052091CA049F
:1025E0003091CB044091CC045091CD040E947729C6
:1025F00029E23CE54FE05EE30E942B2B1816FCF429
:10260000809129058823D9F080911B0590911C05A4
:10261000059790931C0580931B0597FF04C01092AB
:102620001C0510921B050E943D0D80918B0588238F
:1026300031F085E696E064E772E00E9464298091BB
:10264000000590910105A0910205B09103058093CA
:102650000C0590930D05A0930E05B0930F05DF9127
:10266000CF911F910F91FF90EF90DF90CF90BF908F
:10267000AF909F908F907F906F905F904F903F9022
:102680002F9008958091000590910105A091020579
:10269000B09103058093230590932405A09325050D
:1026A000B09326058091BA049091BB04A091BC041C
:1026B000B091BD04805D9740A040B040F1F485E04A
:1026C00060E070E00E94CB2388E060E00E946A2412
:1026D00087E061E00E946A2484E061E00E946A244D
:1026E00088EC90E0A0E0B0E08093BA049093BB0443
:1026F000A093BC04B093BD042EC0809142058823F2
:1027000021F088E061E00E946A24809143058823DB
:1027100021F087E060E00E946A24809144058823CC
:1027200021F084E060E00E946A2460911B057091B2
:102730001C0585E00E94CB2380ED97E0A0E0B0E08F
:102740008093BA049093BB04A093BC04B093BD04DF
:1027500081E0809327058091BE049091BF04A091F1
:10276000C004B091C1042091000530910105409151
:10277000020550910305820F931FA41FB51F80937C
:10278000080590930905A0930A05B0930B051092D4
:102790000C0510920D0510920E0510920F0508956C
:1027A0006F927F928F929F92AF92BF92CF92DF9261
:1027B000EF92FF920F931F93809100059091010576
:1027C000A0910205B0910305809308059093090537
:1027D000A0930A05B0930B058EE00E94A9232091D7
:1027E000490530914A05280F391F30934A05209337
:1027F000490500914B0510914C058FE00E94A923DB
:10280000080F191F10934C0500934B0500914D05BF
:1028100010914E0580E10E94A923080F191F109303
:102820004E0500934D0581E10E94A9237C01809112
:102830004F05909150058E0D9F1D909350058093EC
:102840004F0582E10E94A9235C018091510590917E
:1028500052058A0D9B1D90935205809351058091DE
:102860004505909146050196909346058093450550
:102870000027F7FC0095102FC801B7010E947B2AA2
:1028800020E030EC4FE754E40E94E0292FE632E1EB
:1028900043E850E40E942F2B3B014C01CC24B7FCB1
:1028A000C094DC2CC601B5010E947B2A20E030ECEC
:1028B0004FE754E40E94E0292FE632E143E850E478
:1028C0000E942F2B27E53FE348E65EE30E94E029C4
:1028D0007B018C01C401B3012FEF35EE42E95EE3C9
:1028E0000E94E0299B01AC01C801B7010E942B2B7B
:1028F000181634F48091ED04882311F40E945304D7
:102900001F910F91FF90EF90DF90CF90BF90AF900D
:102910009F908F907F906F90089580910005909187
:102920000105A0910205B0910305809310059093D5
:102930001105A0931205B093130585E696E061E8B2
:1029400072E00E9467288091E5049091E60481304E
:10295000910529F485E696E063E872E00EC00097E1
:1029600029F485E696E06BE872E007C08F5F9F4F21
:1029700031F485E696E065E972E00E94672860918F
:102980008E0570918F058091900590919105209111
:10299000DD043091DE044091DF045091E0040E9498
:1029A000E02920E030E048EC52E40E942F2B0E9406
:1029B000482A9B01AC0185E696E0B9014AE050E067
:1029C0000E94352885E696E06EE972E00E9467284D
:1029D00080912805882331F085E696E060EA72E070
:1029E0000E94672885E696E06AEA72E00E946728FE
:1029F00080912805882309F4D2C040917705509131
:102A000078056091790570917A0585E696E022E077
:102A100030E00E944E2985E696E062EB72E00E946B
:102A2000672840917B0550917C0560917D057091F0
:102A30007E0585E696E022E030E00E944E2985E69C
:102A400096E062EB72E00E94672840917F0550910A
:102A50008005609181057091820585E696E022E00F
:102A600030E00E944E2985E696E064EB72E00E9419
:102A700067284091670550916805609169057091DC
:102A80006A0585E696E022E030E00E944E2985E660
:102A900096E062EB72E00E94672840916B055091CE
:102AA0006C0560916D0570916E0585E696E022E0FB
:102AB00030E00E944E2985E696E062EB72E00E94CB
:102AC000672840916F055091700560917105709174
:102AD000720585E696E022E030E00E944E2985E608
:102AE00096E06BEB72E00E94672880914205882394
:102AF00029F085E696E060EC72E004C085E696E099
:102B000062EC72E00E94672880914305882329F0D7
:102B100085E696E060EC72E004C085E696E062EC43
:102B200072E00E94672880914405882329F085E699
:102B300096E060EC72E004C085E696E062EC72E03C
:102B40000E94672880911A05882331F085E696E077
:102B500064EC72E00E94672885E696E066EC72E01D
:102B60000E946728409183055091840560918505F6
:102B70007091860585E696E022E030E00E944E29BD
:102B800085E696E06CEC72E00E9467284091730540
:102B900050917405609175057091760544C040911F
:102BA0005705509158056091590570915A0585E671
:102BB00096E022E030E00E944E2985E696E062EB46
:102BC00072E00E94672840915B0550915C0560911E
:102BD0005D0570915E0585E696E022E030E00E949A
:102BE0004E2985E696E062EB72E00E9467284091EC
:102BF0005F0550916005609161057091620585E601
:102C000096E022E030E00E944E2985E696E062EDF3
:102C100072E00E94672840916305509164056091BD
:102C200065057091660585E696E022E030E00E9439
:102C30004E2985E696E067ED72E00E946728609174
:102C40001B0570911C0585E696E04AE050E00E9465
:102C5000352885E696E06DED72E00E946728809148
:102C60002805882349F04091870550918805609197
:102C7000890570918A0508C040915305509154050B
:102C8000609155057091560585E696E022E030E0AA
:102C90000E944E2985E696E064EE72E00E94672865
:102CA00060918E0570918F058091900590919105AE
:102CB0000E94482A9B01AC0185E696E0B9014AE0F2
:102CC00050E00E94352885E696E06AEE72E00E94A8
:102CD00067284091E1045091E2046091E30470910F
:102CE000E40485E696E022E030E00E944E2980E090
:102CF00090E0A6ECB2E48093E1049093E204A09308
:102D0000E304B093E40485E696E06FEE72E00E947F
:102D100067284091B1055091B2056091B30570915B
:102D2000B40585E696E022E030E00E944E2985E673
:102D300096E064EF72E00E9467288091ED0488239A
:102D400029F085E696E062EC72E004C085E696E044
:102D500060EC72E00E94672885E696E069EF72E019
:102D60000E94672860918C0570918D0585E696E03C
:102D70004AE050E00E94352885E696E067E671E07B
:102D80000E94642908950F931F93CF93DF93C091FE
:102D9000C105D091C205C133D105E1F485E696E0C5
:102DA0006EEF72E00E94642980914205882349F009
:102DB00085E696E06FEF72E00E94642981E090E082
:102DC0003DC085E696E06AE073E00E94642981E0F8
:102DD00090E03EC0C233D105E1F485E696E06EEFA7
:102DE00072E00E94642980914305882349F085E6BA
:102DF00096E064E173E00E94642982E090E01EC0E6
:102E000085E696E06FE173E00E94642982E090E03D
:102E10001FC0C333D10501F585E696E06EEF72E081
:102E20000E94642980914405882351F085E696E04C
:102E300069E273E00E94642983E090E060E009C0E9
:102E400085E696E064E373E00E94642983E090E005
:102E500061E00E94780499C1C033D10529F588E06A
:102E600060E00E946A2487E061E00E946A2484E0B6
:102E700061E00E946A2485E696E06EEF72E00E94AF
:102E8000642985E696E06EE373E00E94642985E696
:102E900096E06EEF72E00E94642910924205109253
:102EA000430510924405F6C1C136D105F9F485E019
:102EB00060E070E00E94CB2385E696E06EEF72E062
:102EC0000E94642985E696E06DE473E00E9464291F
:102ED00085E696E06EEF72E00E94642910921C0570
:102EE00010921B0585E060E070E0A8C1C236D105F4
:102EF00009F585E064E670E00E94CB2385E696E064
:102F00006EEF72E00E94642985E696E069E573E061
:102F10000E94642985E696E06EEF72E00E946429C3
:102F200084E690E090931C0580931B0585E064E6A1
:102F300070E084C1C336D10509F585E068EC70E026
:102F40000E94CB2385E696E06EEF72E00E94642932
:102F500085E696E067E673E00E94642985E696E0E0
:102F60006EEF72E00E94642988EC90E090931C055B
:102F700080931B0585E068EC70E060C1C436D10524
:102F800009F585E06FEF70E00E94CB2385E696E0BF
:102F90006EEF72E00E94642985E696E065E773E0D3
:102FA0000E94642985E696E06EEF72E00E94642933
:102FB0008FEF90E090931C0580931B0585E06FEFE9
:102FC00070E03CC1C536D105F9F485E696E06EEFB8
:102FD00072E00E94642980911805882349F01092BC
:102FE000180585E696E063E873E00E946728CDC087
:102FF00081E08093180585E696E060E973E00E9421
:1030000067280E943D0DC1C0C636D10569F585E629
:1030100096E06EEF72E00E94642980911905882382
:1030200049F01092190585E696E06CE973E00E947C
:1030300067280BC081E08093190585E696E068EA71
:1030400073E00E9467280E943D0D85E696E06EEFD2
:1030500072E00E94642910920C0510920D051092E6
:103060000E0510920F0516C1C937D10509F56091FB
:10307000B4047091B5048091B6049091B7042DEC1E
:103080003CEC4CE45DE30E9478296093B4047093B7
:10309000B5048093B6049093B70485E696E06EEF8E
:1030A00072E00E94642985E696E063EB73E06BC0F2
:1030B000C836D10509F56091B4047091B5048091CA
:1030C000B6049091B7042DEC3CEC4CE45DE30E9417
:1030D00077296093B4047093B5048093B6049093F9
:1030E000B70485E696E06EEF72E00E94642985E6FB
:1030F00096E065EC73E047C0C537D10509F56091EE
:10310000B0047091B1048091B2049091B3042AE0AC
:1031100037ED43EA5CE30E9478296093B004709332
:10312000B1048093B2049093B30485E696E06EEF09
:1031300072E00E94642985E696E067ED73E023C0A3
:10314000CA36D10549F56091B0047091B1048091FF
:10315000B2049091B3042AE037ED43EA5CE30E94A5
:1031600077296093B0047093B1048093B204909374
:10317000B30485E696E06EEF72E00E94642985E66E
:1031800096E06AEE73E00E94642985E696E06EEFB1
:1031900072E00E9464297EC0C936D10531F585E60A
:1031A00096E06EEF72E00E94642985E696E06FEF8C
:1031B00073E00E94642985E696E06EEF72E00E945B
:1031C000642980911B0590911C050A9690931C051B
:1031D00080931B058F3F910561F15CF18FEF90E0CB
:1031E00090931C0580931B0524C0CB36D10549F56F
:1031F00085E696E06EEF72E00E94642985E696E02F
:103200006AE074E00E94642985E696E06EEF72E061
:103210000E94642980911B0590911C050A97909348
:103220001C0580931B0597FF04C010921C0510928B
:103230001B0560911B0570911C0585E00E94CB2346
:1032400029C0CF36D10531F585E696E06EEF72E004
:103250000E94642985E696E065E174E00E94642995
:1032600085E696E06EEF72E00E94642980911B056E
:1032700090911C05019690931C0580931B058F3F30
:10328000910561F15CF18FEF90E090931C058093C4
:103290001B0524C0CC36D10549F585E696E06EEFD6
:1032A00072E00E94642985E696E06FE174E00E9476
:1032B000642985E696E06EEF72E00E9464298091B1
:1032C0001B0590911C05019790931C0580931B058D
:1032D00097FF04C010921C0510921B0560911B05FE
:1032E00070911C0585E00E94CB237EC1C736D105B5
:1032F00021F585E696E06EEF72E00E9464298091E8
:103300002905882349F085E696E06EE172E00E9487
:1033100064290E9491050CC085E696E064E072E0A5
:103320000E94642960E070E080E090E00E94620A00
:1033300085E696E06EEF72E055C1CA37D10519F403
:103340000E94870751C1C637D10599F48091DA04EC
:10335000882339F01092DA0485E696E069E274E099
:1033600041C181E08093DA0485E696E066E374E08B
:1033700039C1C837D10529F485E696E062E474E0E6
:1033800031C1C137D10559F480918B05882319F0DB
:1033900010928B0529C181E080938B0525C1C2372E
:1033A000D10519F40E9468071FC1C437D10519F46B
:1033B0000E94690419C1CD36D10519F40E94530445
:1033C00013C1CE36D10519F40E9442040DC1C03795
:1033D000D10519F40E94BB0807C1C737D105A9F46C
:1033E0008091000590910105A0910205B09103051F
:1033F000805A9541AF4FBF4F80939C0590939D0598
:10340000A0939E05B0939F05EFC0C337D10509F483
:1034100049C0C433D105E9F480E090E00E949A05E8
:10342000C6E0D0E007C083ED95E0BE0140E00E9419
:10343000B02221968091DB049091DC0401968C17D8
:103440009D078CF786E090E09093DC048093DB048A
:1034500029C0C234D10519F40E94A60623C0C33482
:10346000D10519F580918C0590918D05019787976D
:10347000C8F48091DB049091DC04069799F080E019
:1034800090E00E949A056091DB047091DC04625028
:1034900070407093DC046093DB0483ED95E040E0C2
:1034A0000E94B0220E940E059FC0C533D105E9F4E9
:1034B0008091C5056091C3050E94DE26A0E0B0E0C2
:1034C000BC01CD010E94792A6093DD047093DE0473
:1034D0008093DF049093E0040E94482ADC01CB0132
:1034E00062E070E00E94BD0203C0C633D105C9F49A
:1034F00085E696E064E574E00E9467284091DD046B
:103500005091DE046091DF047091E00485E696E05E
:1035100022E030E00E944E2985E696E067E671E001
:1035200061C0C733D10519F40E94B6025DC0C8332B
:10353000D10591F4C0E0D0E083ED95E0BE0140E01C
:103540000E94B022219682E0C030D807A9F785E614
:1035500096E063E674E046C0C933D105E1F46091BA
:10356000C3058091D1059091D205039719F080E0B1
:1035700090E004C08091C5059091C6050E94DE26AA
:103580008C010E949A050430110571F585E696E0DC
:1035900068EC71E027C0C134D10531F560918E052A
:1035A00070918F0580919005909191050E94482A15
:1035B000DC01CB0160E070E00E94BD02809100055B
:1035C00090910105A0910205B091030580939205A9
:1035D00090939305A0939405B093950585E696E0A6
:1035E00063E774E00E946429DF91CF911F910F91EE
:1035F0000895DF93CF9300D0CDB7DEB7809100055B
:1036000090910105A0910205B091030580930405F6
:1036100090930505A0930605B093070580912805B2
:10362000882309F071C085E696E06FE572E00E949C
:103630000F274091530550915405609155057091A5
:10364000560585E696E022E030E00E94512985E6A5
:1036500096E065E572E00E940F2740915705509172
:1036600058056091590570915A0585E696E022E06B
:1036700030E00E94512985E696E06BE472E00E94FA
:103680000F2740915B0550915C0560915D0570913D
:103690005E0585E696E022E030E00E94512985E64D
:1036A00096E061E472E00E940F2740915F0550911F
:1036B0006005609161057091620585E696E022E003
:1036C00030E00E94512985E696E063E372E00E94B3
:1036D0000F27609157057091580580915905909179
:1036E0005A0520915B0530915C0540915D05509134
:1036F0005E050E94782920915F0530916005409118
:10370000610550916205D6C085E696E06BE172E0F6
:103710000E940F2740918705509188056091890587
:1037200070918A0585E696E022E030E00E945129FA
:1037300085E696E068E072E00E940F2740917705E9
:10374000509178056091790570917A0585E696E04B
:1037500022E030E00E94512985E696E065EF71E0B5
:103760000E940F2740917B0550917C0560917D055B
:1037700070917E0585E696E022E030E00E945129B6
:1037800085E696E062EE71E00E940F2740917F058A
:1037900050918005609181057091820585E696E0E3
:1037A00022E030E00E94512985E696E06BEC71E062
:1037B0000E940F27609177057091780580917905B7
:1037C00090917A0520917B0530917C0540917D0593
:1037D00050917E050E94782920917F0530918005C7
:1037E00040918105509182050E947829AB01BC016E
:1037F00085E696E022E030E00E94512985E696E0D9
:103800006CEB71E00E940F274091670550916805AD
:103810006091690570916A0585E696E022E030E0E6
:103820000E94512985E696E06DEA71E00E940F271B
:1038300040916B0550916C0560916D0570916E051E
:1038400085E696E022E030E00E94512985E696E088
:103850006EE971E00E940F2740916F05509170054D
:10386000609171057091720585E696E022E030E086
:103870000E94512985E696E06BE871E00E940F27CF
:1038800060916705709168058091690590916A055E
:1038900020916B0530916C0540916D0550916E053E
:1038A0000E94782920916F05309170054091710533
:1038B000509172050E947829AB01BC0185E696E023
:1038C00022E030E00E94512985E696E062E871E04E
:1038D0000E940F2760911B0570911C0585E696E0FC
:1038E0004AE050E00E94482885E696E063E771E0F0
:1038F0000E940F274091B0045091B1046091B2042E
:103900007091B30485E696E022E030E00E945129F0
:1039100085E696E065E671E00E940F274091B404C9
:103920005091B5046091B6047091B70485E696E0B5
:1039300022E030E00E94512980914205882311F451
:1039400090E007C085E696E066E571E00E940F27EB
:1039500091E080914305882339F085E696E067E49D
:1039600071E00E940F2791E080914405882339F08F
:1039700085E696E068E371E00E940F2791E0809170
:103980001805882339F085E696E06BE271E00E9425
:103990000F2791E080911905882339F085E696E09C
:1039A0006FE171E00E940F2791E080911A05882352
:1039B00039F085E696E064E171E00E940F2702C0CD
:1039C000992331F085E696E06EEF72E00E9464295B
:1039D00085E696E062E171E00E940F2740910005C4
:1039E00050910105609102057091030585E696E00E
:1039F0002AE030E00E94E62785E696E060E171E08B
:103A00000E940F2780912805882309F445C0409122
:103A10008705509188056091890570918A0585E632
:103A200096E022E030E00E944E2985E696E06EE0C6
:103A300071E00E940F2740917705509178056091C1
:103A4000790570917A0585E696E022E030E00E94E3
:103A50004E2985E696E06CE071E00E940F274091C8
:103A60007B0550917C0560917D0570917E0585E612
:103A700096E022E030E00E944E2985E696E06AE07A
:103A800071E00E940F2740917F0550918005609161
:103A900081057091820544C04091530550915405B1
:103AA000609155057091560585E696E022E030E07C
:103AB0000E944E2985E696E068E071E00E940F279B
:103AC00040915705509158056091590570915A05DC
:103AD00085E696E022E030E00E944E2985E696E0F9
:103AE00066E071E00E940F2740915B0550915C05F4
:103AF00060915D0570915E0585E696E022E030E01C
:103B00000E944E2985E696E064E071E00E940F274E
:103B100040915F055091600560916105709162056B
:103B200085E696E022E030E00E944E2985E696E0A8
:103B300062E071E00E940F27409163055091640597
:103B4000609165057091660585E696E022E030E0BB
:103B50000E944E2985E696E060E071E00E940F2702
:103B600060911B0570911C0585E696E04AE050E0E7
:103B70000E94352885E696E06EEF70E00E9452279D
:103B800085E696E060EF70E00E940F2760914705A0
:103B90007091480585E696E04AE050E00E9448288A
:103BA00085E696E06DED70E00E940F274091B1052B
:103BB0005091B2056091B3057091B40585E696E029
:103BC00022E030E00E9451298091ED04882329F001
:103BD00085E696E06DEC70E004C085E696E06EEB5D
:103BE00070E00E94522780912805882319F185E60C
:103BF00096E06DEA70E00E940F27409173055091A6
:103C00007405609175057091760585E696E022E071
:103C100030E00E94512985E696E068E970E00E9454
:103C20000F2740918305509184056091850570911F
:103C300086050EC085E696E06CE870E00E940F27CE
:103C4000409163055091640560916505709166052A
:103C500085E696E022E030E00E94512980918C05B3
:103C600090918D05892B81F085E696E064E870E0FF
:103C70000E940F2760918C0570918D0585E696E076
:103C80004AE050E00E94482885E696E069E770E047
:103C90000E940F278091870690918806009711F463
:103CA0008BE896E0BE016F5F7F4F681B790B85E65E
:103CB00096E04AE050E00E94482885E696E06EEFE4
:103CC00072E00E9464290F900F90CF91DF910895C8
:103CD00085E696E00E940F269C014091D105509107
:103CE000D205FA01EE0FFF1FEF53FA4F9183808345
:103CF000BA016F5F7F4F7093D2056093D1058D300D
:103D0000910519F08A30910571F48091C105909167
:103D1000C205C59741F0161617062CF45093D2052C
:103D20004093D10509C08091C1059091C205C59706
:103D300031F46330710519F40E94C31609C02D30A7
:103D4000310519F02A30310539F46130710521F45B
:103D50001092D2051092D105809100059091010535
:103D6000A0910205B09103058093A9059093AA053F
:103D7000A093AB05B093AC0580918C0590918D0517
:103D8000479709F040C080E090E00E949A058DECD2
:103D90009CECA4E8B0E48093C6049093C704A0937D
:103DA000C804B093C90483E393E3A3E8B0E4809329
:103DB000320590933305A0933405B093350583E322
:103DC00093E3A3E7B0E48093D6049093D704A09341
:103DD000D804B093D9048DEC9CECACE4B0E48093AF
:103DE000E9049093EA04A093EB04B093EC0480E020
:103DF00090E0A0E8BFE38093CA049093CB04A09323
:103E0000CC04B093CD040895AF92BF92CF92DF92CD
:103E1000EF92FF920F931F930E9404230E94792A2E
:103E200020E030E040E85CE30E942F2B0E944D2A06
:103E30005B016C018091000590910105A091020544
:103E4000B0910305A816B906CA06DB0640F4A09295
:103E50001F05B0922005C0922105D0922205A092A4
:103E60000005B0920105C0920205D0920305809131
:103E700042058823D9F4809143058823B9F48091C1
:103E80004405882399F480911B0590911C05181610
:103E9000190664F080911805882341F48091190572
:103EA000882321F480912905882321F081E08093E3
:103EB000280502C010922805E090BA04F090BB04D7
:103EC0000091BC041091BD04A60195012E193F0973
:103ED000400B510B8091230590912405A09125055D
:103EE000B091260582179307A407B50758F4AE14BE
:103EF000BF04C006D10630F080912805882311F058
:103F00000E944213E0900005F09001050091020527
:103F100010910305A80197012A5F304040405040AE
:103F200080910C0590910D05A0910E05B0910F05A3
:103F300082179307A407B507F8F42AEFE216F104F5
:103F400001051105C8F080914505909146051816A8
:103F5000190694F40E9457100E949C0A0E94D902EC
:103F60000E94DF080E948F080E9456080E943907AD
:103F70000E940B070E94DA06E0900005F090010510
:103F80000091020510910305A8019701205D3740BB
:103F9000404050408091040590910505A091060590
:103FA000B091070582179307A407B507E0F480EDE9
:103FB000E81687E0F80680E0080780E0180798F028
:103FC0008091BA049091BB04A091BC04B091BD044F
:103FD000883C9105A105B10531F080918B058823BE
:103FE00011F00E94F91AE0900005F090010500918F
:103FF000020510910305A80197012A5F3040404057
:1040000050408091140590911505A0911605B0912E
:10401000170582179307A407B50780F42AEFE21665
:10402000F1040105110550F080911805882321F451
:1040300080911905882311F00E94AD0BE0900005D6
:10404000F09001050091020510910305A801970168
:10405000245C39404040504080912A0590912B05C6
:10406000A0912C05B0912D0582179307A407B507E1
:1040700078F484ECE81689E0F80680E0080780E030
:10408000180730F080912905882311F00E94A50EB1
:10409000E0900005F09001050091020510910305E4
:1040A000A8019701285833414040504080911005A5
:1040B00090911105A0911205B091130582179307F5
:1040C000A407B507E0F428E8E21623E1F20620E0B1
:1040D000020720E0120798F08091BA049091BB0487
:1040E000A091BC04B091BD04883C9105A105B10527
:1040F00031F080918B05882311F40E948D14E0909B
:104100000005F09001050091020510910305A8013A
:104110009701205E33494440504080919205909130
:104120009305A0919405B091950582179307A40774
:10413000B50708F580EEE81683E9F80684E008077D
:1041400080E01807C0F0E0929205F092930500938A
:1041500094051093950560918E0570918F0580915F
:104160009005909191050E94482ADC01CB0160E006
:1041700070E00E94BD022091B5053091B6054091D6
:10418000B7055091B8058091000590910105A09167
:104190000205B0910305281739074A075B0738F471
:1041A000211531054105510511F00E9487078091C5
:1041B000BF059091C0050E943003E0900005F0908B
:1041C00001050091020510910305A80197012058EF
:1041D0003F44424150408091A9059091AA05A09189
:1041E000AB05B091AC0582179307A407B507A8F4F7
:1041F00020E8E2162FE4F20622E1020720E012078F
:1042000060F0E092A905F092AA050093AB05109327
:10421000AC0587E190E00E949A058091000590919D
:104220000105A0910205B091030520911F05309171
:1042300020054091210550912205821B930BA40B70
:10424000B50B815C944DA140B04040F080911A05BF
:10425000882321F08CE290E00E949A05A09000054E
:10426000B0900105C0900205D0900305E090AC0429
:10427000F090AD040091AE041091AF04A601950139
:104280002E193F09400B510B8091080590910905AB
:10429000A0910A05B0910B0582179307A407B507F3
:1042A00038F4AE14BF04C006D10610F00E94D0133B
:1042B00085E696E00E94DE25181619067CF48091AA
:1042C000BA049091BB04A091BC04B091BD04883C99
:1042D0009105A105B10511F00E94681E20919C0571
:1042E00030919D0540919E0550919F052115310506
:1042F0004105510579F18091000590910105A0914A
:104300000205B091030582179307A407B50710F1C2
:1043100060918E0570918F05809190059091910527
:104320000E94482ADC01CB0160E070E00E94BD02DF
:104330000E94B3040E94680785E696E067E874E08F
:104340000E94642910929C0510929D0510929E0572
:1043500010929F051F910F91FF90EF90DF90CF90EB
:10436000BF90AF900895AF92BF92CF92DF92EF923D
:10437000FF920F931F9380E00E94A6238EE060E0DF
:104380000E942B248FE060E00E942B2480E160E0FB
:104390000E942B2481E160E00E942B2482E160E0F6
:1043A0000E942B2488E061E00E942B2487E061E0DA
:1043B0000E942B2484E061E00E942B2488E060E0CE
:1043C0000E946A2487E061E00E946A2484E061E040
:1043D0000E946A2485B5887F816085BD8DE061E09B
:1043E0000E942B248DE06091BF050E946A2485E025
:1043F00061E00E942B2460911B0570911C0585E0F3
:104400000E94CB2383E061E00E942B2483E061E0E3
:104410000E946A2482E061E00E942B2482E060E036
:104420000E946A2485E696E040E052EC61E070E08C
:104430000E94572585E696E066E974E00E946429AB
:1044400082E090E00E94F0049C01181619067CF4AA
:10445000B901882777FD8095982F0E947B2A609369
:10446000DD047093DE048093DF049093E00480E029
:1044700090E00E94F004AA2797FDA095BA2FBC01F6
:10448000CD010E947B2A5B016C01E090DD04F0907D
:10449000DE040091DF041091E004A80197010E945E
:1044A0002B2B18164CF4E0928E05F0928F0500939A
:1044B00090051093910508C0A0928E05B0928F05CB
:1044C000C0929005D092910584E090E00E94F004A3
:1044D0009C01009771F1285E3340B901882777FD70
:1044E0008095982F0E947B2A20E030E04AE754E430
:1044F0000E94E0296093B1057093B2058093B305E3
:104500009093B40516C00E94F0040097C9F09093F0
:104510008D0580938C058731910511F00E949A05D5
:104520008091DB049091DC0402969093DC048093EC
:10453000DB048091DB049091DC048D3191051CF348
:104540001F910F91FF90EF90DF90CF90BF90AF90B1
:104550000895F999FECF72BD61BDF89A80B50895AE
:10456000F999FECF1FBA72BD61BD40BD0FB6F89478
:10457000FA9AF99A0FBE08951F920F920FB60F92F2
:1045800011242F933F938F939F93AF93BF93809169
:10459000D8059091D905A091DA05B091DB0530914D
:1045A000DC050196A11DB11D232F2D5F2D3720F0B5
:1045B0002D570196A11DB11D2093DC058093D805D0
:1045C0009093D905A093DA05B093DB058091D405CB
:1045D0009091D505A091D605B091D7050196A11D62
:1045E000B11D8093D4059093D505A093D605B093C3
:1045F000D705BF91AF919F918F913F912F910F90D0
:104600000FBE0F901F9018958FB7F8942091D80582
:104610003091D9054091DA055091DB058FBFB90182
:10462000CA0108959B01AC017FB7F8948091D4052D
:104630009091D505A091D605B091D70566B5A89BF8
:1046400005C06F3F19F00196A11DB11D7FBFBA2FA4
:10465000A92F982F8827860F911DA11DB11D62E0FB
:10466000880F991FAA1FBB1F6A95D1F7BC012DC0E7
:10467000FFB7F8948091D4059091D505A091D60507
:10468000B091D705E6B5A89B05C0EF3F19F001969C
:10469000A11DB11DFFBFBA2FA92F982F88278E0FFC
:1046A000911DA11DB11DE2E0880F991FAA1FBB1F1C
:1046B000EA95D1F7861B970B885E9340C8F221508C
:1046C00030404040504068517C4F21153105410534
:1046D000510571F60895789484B5826084BD84B5DF
:1046E000816084BD85B5826085BD85B5816085BDED
:1046F000EEE6F0E0808181608083E1E8F0E0108206
:10470000808182608083808181608083E0E8F0E046
:10471000808181608083E1EBF0E080818460808330
:10472000E0EBF0E0808181608083EAE7F0E0808167
:1047300084608083808182608083808181608083C7
:104740008081806880831092C10008958093EE0478
:104750000895982F8E3008F09E5097708091EE0447
:104760008295880F880F807C892B80937C008091B4
:104770007A00806480937A0080917A0086FDFCCF75
:104780002091780040917900942F80E030E0282B30
:10479000392BC90108951F93CF93DF93182FEB0195
:1047A00061E00E942B24209709F44AC0CF3FD10535
:1047B00009F449C0E12FF0E0EC54FD4F84918330BF
:1047C000C1F0843028F4813051F08230B1F50CC052
:1047D000863019F1873049F1843079F514C084B5F9
:1047E000806884BDC7BD33C084B5806284BDC8BD48
:1047F0002EC080918000806880938000D0938900D3
:10480000C093880024C080918000806280938000E3
:10481000D0938B00C0938A001AC08091B00080684A
:104820008093B000C093B30012C08091B00080624A
:104830008093B000C093B4000AC0C038D1051CF406
:10484000812F60E002C0812F61E00E946A24DF9125
:10485000CF911F910895CF93DF93482F50E0CA0165
:1048600080569D4FFC01349144575D4FFA0184916D
:10487000882369F190E0880F991FFC01E259FD4FF0
:10488000A591B491FC01E858FD4FC591D4916623E0
:1048900051F42FB7F8948C91932F909589238C9392
:1048A000888189230BC0623061F42FB7F8948C9112
:1048B000932F909589238C938881832B88832FBF96
:1048C00006C09FB7F8948C91832B8C939FBFDF9188
:1048D000CF910895482F50E0CA018C549D4FFC01A0
:1048E0002491CA0180569D4FFC01949144575D4F1D
:1048F000FA013491332309F440C0222351F12330CB
:1049000071F0243028F42130A1F0223011F514C0C8
:104910002630B1F02730C1F02430D9F404C08091A2
:1049200080008F7703C0809180008F7D809380000E
:1049300010C084B58F7702C084B58F7D84BD09C057
:104940008091B0008F7703C08091B0008F7D8093FD
:10495000B000E32FF0E0EE0FFF1FE858FD4FA591E8
:10496000B4912FB7F894662321F48C919095892304
:1049700002C08C91892B8C932FBF0895CF93DF9326
:104980000E946B230E94B321C9E0D5E20E94041F5C
:104990002097E1F30E940925F9CF08951F920F9205
:1049A0000FB60F9211242F933F934F938F939F93A2
:1049B000EF93FF938091C00082FD1DC04091C6001F
:1049C00020911D0630911E062F5F3F4F2F733070D0
:1049D00080911F06909120062817390771F0E09109
:1049E0001D06F0911E06E352FA4F408330931E06D7
:1049F00020931D0602C08091C600FF91EF919F9108
:104A00008F914F913F912F910F900FBE0F901F905C
:104A10001895E0917106F0917206E05CFF4F81916C
:104A2000919120813181821B930B8F739070892B20
:104A300011F00E94CD2408951F920F920FB60F928D
:104A400011242F933F938F939F93EF93FF93209184
:104A50006106309162068091630690916406281782
:104A6000390731F48091C1008F7D8093C10014C05B
:104A7000E0916306F0916406EF5DF94F208180912B
:104A800063069091640601968F739070909364060C
:104A9000809363062093C600FF91EF919F918F91C1
:104AA0003F912F910F900FBE0F901F901895AF92CE
:104AB000BF92DF92EF92FF920F931F93CF93DF93FA
:104AC000EC017A018B01DD24403081EE580780E053
:104AD000680780E0780711F0DD24D39491E0A92ED7
:104AE000B12CEC89FD89DD2069F0C50108A002C068
:104AF000880F991F0A94E2F7808360E079E08DE3E4
:104B000090E005C0108260E874E88EE190E0A801B2
:104B100097010E94C82B215030404040504056958C
:104B200047953795279580E12030380720F0DD2024
:104B300011F0DD24D6CFE889F9893083EA89FB8931
:104B4000208319A2EE89FF89408121E030E0C9016C
:104B50000C8C02C0880F991F0A94E2F7482B4083FF
:104B6000EE89FF894081C9010D8C02C0880F991F11
:104B70000A94E2F7482B4083EE89FF894081C901FE
:104B80000E8C02C0880F991F0A94E2F7482B4083CD
:104B9000EE89FF8980810F8C02C0220F331F0A9497
:104BA000E2F7209528232083DF91CF911F910F9169
:104BB000FF90EF90DF90BF90AF900895DC011C96BE
:104BC000ED91FC911D97E05CFF4F21913191808127
:104BD0009181281B390B2F733070C9010895DC01B6
:104BE0001C96ED91FC911D97E05CFF4F2081318177
:104BF000E054F040DF01AE5BBF4F8D919C91119767
:104C00002817390719F42FEF3FEF07C08D919C91BA
:104C1000E80FF91F8081282F30E0C9010895DC01D9
:104C20001C96ED91FC911D97E05CFF4F2081318136
:104C3000E054F040DF01AE5BBF4F8D919C91119726
:104C40002817390719F42FEF3FEF10C08D919C9171
:104C50001197E80FF91F20818D919C911197019672
:104C60008F73907011969C938E9330E0C9010895D4
:104C7000DC0191968C919197882339F05496ED91AF
:104C8000FC915597808186FFF9CF91961C920895EB
:104C9000CF93DF93EC01EE85FF85E05CFF4F208131
:104CA0003181E054F0402F5F3F4F2F733070DF01B0
:104CB000AE5BBF4F8D919C91119728173907D1F3A7
:104CC000E05CFF4F80819181E054F040E80FF91FD4
:104CD0006083EE85FF85E05CFF4F31832083EE89A2
:104CE000FF89208181E090E00F8C02C0880F991F1E
:104CF0000A94E2F7282B208381E089A3EC89FD89BF
:104D000080818064808381E090E0DF91CF9108957D
:104D1000109268061092670688EE93E0A0E0B0E07B
:104D20008093690690936A06A0936B06B0936C0615
:104D300083EF94E090936606809365068DED95E091
:104D4000909372068093710681E296E090937406C8
:104D50008093730685EC90E09093760680937506B9
:104D600084EC90E0909378068093770680EC90E056
:104D700090937A068093790681EC90E090937C067C
:104D800080937B0682EC90E090937E0680937D0674
:104D900086EC90E09093800680937F0684E0809379
:104DA000810683E08093820687E08093830685E016
:104DB0008093840681E080938506089570E0382F03
:104DC00020E0622B732BCB010895CF92DF92EF92FC
:104DD000FF920F931F93CF93DF937C016B018A01A6
:104DE000C0E0D0E00FC0D6016D916D01D701ED910B
:104DF000FC910190F081E02DC7010995C80FD91FE2
:104E0000015010400115110571F7CE01DF91CF91CE
:104E10001F910F91FF90EF90DF90CF900895EF9248
:104E2000FF920F931F93CF93DF937C018B01C0E020
:104E3000D0E0F8010F5F1F4F6491662359F0D7014E
:104E4000ED91FC910190F081E02DC7010995C80F0B
:104E5000D91FEFCFCE01DF91CF911F910F91FF901E
:104E6000EF900895EF92FF920F931F938C01DC0156
:104E7000ED91FC910190F081E02D6DE009957C01B0
:104E8000D801ED91FC910190F081E02DC8016AE01C
:104E900009959C012E0D3F1DC9011F910F91FF9097
:104EA000EF900895EF92FF920F931F937C010E9461
:104EB0000F278C01C7010E9432279C01200F311F50
:104EC000C9011F910F91FF90EF900895CF93DF9349
:104ED000EC016115710519F420E030E00FC0DB0131
:104EE0000D900020E9F71197A61BB70BE881F98117
:104EF0000280F381E02DAD0109959C01C901DF918C
:104F0000CF9108954F925F927F928F929F92AF922E
:104F1000BF92CF92DF92EF92FF920F931F93DF9396
:104F2000CF93CDB7DEB7A1970FB6F894DEBF0FBE13
:104F3000CDBF2C01742ECB01223008F42AE019A237
:104F400031E2C32ED12CCC0EDD1E822E9924AA2450
:104F5000BB24672D752FA50194010E94C82B7901F0
:104F60008A01C801B701A50194010E94962B472D23
:104F7000461B0894C108D1084A3014F4405D01C0B2
:104F8000495CF6014083E114F1040105110521F0AB
:104F90007E2C5F2DC801DDCFC201B6010E946627BD
:104FA000A1960FB6F894DEBF0FBECDBFCF91DF91B3
:104FB0001F910F91FF90EF90DF90CF90BF90AF9037
:104FC0009F908F907F905F904F900895DC01211506
:104FD000310541F4ED91FC910190F081E02D642FB9
:104FE000099508950E9482270895CF92DF92EF924B
:104FF000FF920F931F93CF93DF93EC016A017B0124
:105000002115310541F4E881F9810190F081E02D0D
:10501000642F09951FC02A303105D1F477FF17C0DE
:10502000E881F9810190F081E02D6DE209958C0114
:1050300044275527BA014C195D096E097F09CE0135
:105040002AE00E9482279801280F391F04C02AE015
:105050000E9482279C01C901DF91CF911F910F917E
:10506000FF90EF90DF90CF900895EF92FF920F9313
:105070001F937B019A010027F7FC0095102FB801C0
:10508000A7010E94F5271F910F91FF90EF900895BF
:10509000CF92DF92EF92FF920F931F936C017B01EF
:1050A0009A010027F7FC0095102FB801A7010E9474
:1050B000F5278C01C6010E943227080F191FC8016D
:1050C0001F910F91FF90EF90DF90CF9008950E9475
:1050D000662708957F928F929F92AF92BF92CF9250
:1050E000DF92EF92FF920F931F93CF93DF934C01C8
:1050F0007A018B01722ECB01BA01A80197010E949F
:10510000922B882321F0C4016EE974E021C0C0E035
:10511000D0E057016801E894D7F8C601B5012FEF38
:105120003FEF4FE75FE70E94922B882351F4C601BF
:10513000B5012FEF3FEF4FE75FE70E94DC2918161C
:1051400014F0C1E0D0E0219739F0C40162EA74E0C4
:105150000E946627EC0193C0C801B7012FEF3FEF13
:105160004FE75FE40E942B2B181654F0C801B701DB
:105170002FEF3FEF4FE75FEC0E94DC29882324F4F8
:10518000C40166EA74E0E4CFC801B70120E030E072
:1051900040E050E00E94DC2987FD03C0C0E0D0E081
:1051A0000EC0D401ED91FC910190F081E02DC4017D
:1051B0006DE20995EC0117FB109517F9109520E0A9
:1051C00030E040E05FE3DD240BC0CA01B90120E01C
:1051D00030E040E251E40E94E0299B01AC01D3940D
:1051E000D71498F3C801B7010E9478295B016C01BC
:1051F0000E944D2A7B018C01C401B801A7012AE05D
:1052000030E00E94E627C80FD91F772039F0C4018B
:105210006AEA74E00E946627C80FD91FC801B70167
:105220000E94792A9B01AC01C601B5010E94772931
:1052300024C020E030E040E251E40E942F2B7B01AB
:105240008C010E94482A5B016C01CC24B7FCC094FD
:10525000DC2CC401B601A5012AE030E00E94F5274C
:10526000C80FD91FC601B5010E947B2A9B01AC0162
:10527000C801B7010E9477297A947720D1F6CE0130
:10528000DF91CF911F910F91FF90EF90DF90CF9022
:10529000BF90AF909F908F907F9008950E946A2852
:1052A0000895EF92FF920F931F937C010E946A284A
:1052B0008C01C7010E943227080F191FC8011F91D6
:1052C0000F91FF90EF900895EF92FF920F931F932D
:1052D0007C010E9466278C01C7010E943227080FBB
:1052E000191FC8011F910F91FF90EF90089550581A
:1052F000BB27AA270ED075C166D130F06BD120F044
:1053000031F49F3F11F41EF45BC10EF4E095E7FB0E
:1053100051C1E92F77D180F3BA1762077307840769
:10532000950718F071F49EF58FC10EF4E0950B2EE1
:10533000BA2FA02D0B01B90190010C01CA01A001E7
:105340001124FF27591B99F0593F50F4503E68F142
:105350001A16F040A22F232F342F4427585FF3CF83
:10536000469537952795A795F0405395C9F77EF454
:105370001F16BA0B620B730B840BBAF09150A1F09D
:10538000FF0FBB1F661F771F881FC2F70EC0BA0F23
:10539000621F731F841F48F4879577956795B795AB
:1053A000F7959E3F08F0B3CF9395880F08F09927A3
:1053B000EE0F979587950895D9D008F481E0089568
:1053C0000CD00FC107D140F0FED030F021F45F3F88
:1053D00019F0F0C0511139C1F3C014D198F39923D9
:1053E000C9F35523B1F3951B550BBB27AA276217A9
:1053F0007307840738F09F5F5F4F220F331F441FEE
:10540000AA1FA9F333D00E2E3AF0E0E830D0915025
:105410005040E695001CCAF729D0FE2F27D0660F12
:10542000771F881FBB1F261737074807AB07B0E851
:1054300009F0BB0B802DBF01FF2793585F4F2AF067
:105440009E3F510568F0B6C000C15F3FECF3983E47
:10545000DCF3869577956795B795F7959F5FC9F7C4
:10546000880F911D9695879597F90895E1E0660F4D
:10547000771F881FBB1F621773078407BA0720F0C6
:10548000621B730B840BBA0BEE1F88F7E09508952F
:1054900004D06894B111D9C00895BCD088F09F574A
:1054A00090F0B92F9927B751A0F0D1F0660F771F70
:1054B000881F991F1AF0BA95C9F712C0B13081F050
:1054C000C3D0B1E00895C0C0672F782F8827B85F98
:1054D00039F0B93FCCF3869577956795B395D9F7B1
:1054E0003EF490958095709561957F4F8F4F9F4FBB
:1054F0000895E89409C097FB3EF4909580957095C7
:1055000061957F4F8F4F9F4F9923A9F0F92F96E90F
:10551000BB279395F695879577956795B795F11184
:10552000F8CFFAF4BB0F11F460FF1BC06F5F7F4F21
:105530008F4F9F4F16C0882311F096E911C0772333
:1055400021F09EE8872F762F05C0662371F096E83C
:10555000862F70E060E02AF09A95660F771F881F0B
:10556000DAF7880F9695879597F90895990F0008AF
:10557000550FAA0BE0E8FEEF16161706E807F90725
:10558000C0F012161306E407F50798F0621B730BC0
:10559000840B950B39F40A2661F0232B242B252B41
:1055A00021F408950A2609F4A140A6958FEF811DE4
:1055B000811D089597F99F6780E870E060E0089585
:1055C0009FEF80EC089500240A941616170618061B
:1055D0000906089500240A941216130614060506F7
:1055E0000895092E0394000C11F4882352F0BB0F88
:1055F00040F4BF2B11F460FF04C06F5F7F4F8F4FEB
:105600009F4F089557FD9058440F551F59F05F3F25
:1056100071F04795880F97FB991F61F09F3F79F0D4
:1056200087950895121613061406551FF2CF469556
:10563000F1DF08C0161617061806991FF1CF8695D8
:105640007105610508940895E894BB2766277727BC
:10565000CB0197F908958ADF08F48FEF08950BD0F6
:10566000C0CFB1DF28F0B6DF18F0952309F0A2CF44
:10567000A7CF1124EACFC6DFA0F3959FD1F3950FF2
:1056800050E0551F629FF001729FBB27F00DB11DC6
:10569000639FAA27F00DB11DAA1F649F6627B00D56
:1056A000A11D661F829F2227B00DA11D621F739F3F
:1056B000B00DA11D621F839FA00D611D221F749F4D
:1056C0003327A00D611D231F849F600D211D822F94
:1056D000762F6A2F11249F5750408AF0E1F08823DB
:1056E0004AF0EE0FFF1FBB1F661F771F881F9150E8
:1056F0005040A9F79E3F510570F05CCFA6CF5F3FA9
:10570000ECF3983EDCF3869577956795B795F7951A
:10571000E7959F5FC1F7FE2B880F911D96958795A2
:1057200097F9089523DF880B990B0895629FD001A4
:10573000739FF001829FE00DF11D649FE00DF11D4C
:10574000929FF00D839FF00D749FF00D659FF00DFB
:105750009927729FB00DE11DF91F639FB00DE11DE8
:10576000F91FBD01CF011124089597FB092E0726CB
:105770000AD077FD04D02ED006D000201AF4709500
:1057800061957F4F0895F6F7909581959F4F089505
:10579000A1E21A2EAA1BBB1BFD010DC0AA1FBB1F35
:1057A000EE1FFF1FA217B307E407F50720F0A21BA7
:1057B000B30BE40BF50B661F771F881F991F1A9414
:1057C00069F760957095809590959B01AC01BD013E
:1057D000CF010895AA1BBB1B51E107C0AA1FBB1F25
:1057E000A617B70710F0A61BB70B881F991F5A956D
:1057F000A9F780959095BC01CD010895EE0FFF1F8C
:0C5800000590F491E02D0994F894FFCF7E
:10580C003C77616C6C706F7765723E00626174748A
:10581C00506C757350696E20484947482028666C57
:10582C006F77290062617474506C757350696E20C7
:10583C004C4F5720286E6F20666C6F772900626181
:10584C007474207361666574792073776974636806
:10585C00204F4E003C706F7765725F6572726F728D
:10586C002000303E002C003E0077726974696E6730
:10587C00206572726F7220746F20656570726F6D27
:10588C00003C666F7263655F756E646F636B3E00A0
:10589C0062617474207361666574792073776974BE
:1058AC006368204F4646000A7A65726F20637572F2
:1058BC0072656E740A006E65772063757272656E20
:1058CC00742063616C3A20003C7265646F636B3EBC
:1058DC00003C73687574646F776E3E0064616E672C
:1058EC0065726F75736C79206C6F772063656C6C67
:1058FC00003C636861726765643E003C646F636B77
:10590C0065643E006175746F206368617267652021
:10591C004F4E003C756E646F636B65643E00617541
:10592C00746F20636861726765204F4646000A6D8C
:10593C006178206368617267652074696D650A001F
:10594C000A707265636F6E646974696F6E696E67F5
:10595C000A003C686967685F63757272656E743EB5
:10596C000068696768204348415247494E472063A5
:10597C00656C6C00686967682063757272656E741B
:10598C00003C00646F636B65642000756E646F632C
:10599C006B65642000756E6B6E6F776E2000250052
:1059AC005F6368617267696E67002063656C6C7316
:1059BC003A005F005F69646C653A005F73683A0097
:1059CC003100300041005F7343563A005F73495613
:1059DC003A005F73563A005F70776D3A005F616D05
:1059EC0070733A005F6D41683A005F6C563A005F25
:1059FC0063433A005F62503A005F65523A000073AD
:105A0C0068756E7431204F4646007368756E74313C
:105A1C00204F4E007368756E7432204F46460073EB
:105A2C0068756E7432204F4E007368756E74332037
:105A3C004F4646007368756E7433204F4E00736882
:105A4C00756E747320616C6C206F666600766F6C7B
:105A5C0074732050574D203000766F6C7473205047
:105A6C00574D2031303000766F6C74732050574D89
:105A7C002032303000766F6C74732050574D2032CA
:105A8C0035350061646A566F6C7473204F4646005E
:105A9C0061646A566F6C7473204F4E0061646A4186
:105AAC006D7073204F46460061646A416D707320BF
:105ABC004F4E0074617267657420416D7073202BBA
:105ACC00302E30350074617267657420416D7073CF
:105ADC00202D302E30350074617267657420766F1E
:105AEC006C7473202B302E303200746172676574C5
:105AFC0020766F6C7473202D302E30323A2000706B
:105B0C00777250574D202B31300070777250574DB3
:105B1C00202D31300070777250574D202B31007092
:105B2C00777250574D202D310066756C6C61757411
:105B3C006F204F46460066756C6C6175746F204F14
:105B4C004E003C69643A3A6F63756C7573506F77AD
:105B5C0065723E003C6D41684361706163697479A4
:105B6C003A20003C656570726F6D5F65726173659C
:105B7C00643E003C77726974696E675F746F5F6531
:105B8C006570726F6D3E003C5348555454494E47F6
:105B9C00444F574E3E003C72657365743E006E6117
:105BAC006E00696E66006F7666002E000A000000BB
:105BBC00333383400000003F0500D0070000320063
:105BCC000000C4090000CDCC84400000803F009749
:105BDC00490160EA00003333734001060000D084B1
:105BEC00450000C642FFFFFFFFCDCC4C4001010039
:105BFC000000004826E526DE250F26EF2538260076
:00000001FF
